:100000000C9446000C9463000C9463000C94630001
:100010000C9463000C9463000C9463000C946300D4
:100020000C9463000C9463000C9463000C946300C4
:100030000C9463000C9463000C9463000C946300B4
:100040000C9490020C9463000C9463000C94630075
:100050000C9463000C9463000C9463000C94630094
:100060000C9463000C9463000C9463000C94630084
:100070000C9463000C9463000C9463000C94630074
:100080000C9463000C94AD000C94630011241FBE0B
:10009000CFEFD0E1DEBFCDBF11E0A0E0B1E0E6EFF1
:1000A000F5E000E00BBF02C007900D92AA32B10745
:1000B000D9F712E0AAE2B1E001C01D92AE36B10755
:1000C000E1F70C9465000C940000CFEFD0E1DEBFA7
:1000D000CDBF0E94C502809164008061809364005E
:1000E00086ED90E00E94CC01882331F48091650078
:1000F000806180936500FFCF789440E050E0443108
:10010000510589F0453151053CF44115510559F02F
:100110004A30510561F013C04E31510541F044366B
:10012000510559F00CC080916500806103C0809139
:1001300065008F7E8093650002C04FEF5FEF4F5FD9
:100140005F4F20912A0130912B0180912A019091DB
:100150002B0182179307C9F3D2CF1F920F920FB6CC
:100160000F9211242F933F934F935F936F937F933D
:100170008F939F93AF93BF93EF93FF930E94C3011D
:1001800080917400806880937400FF91EF91BF911B
:10019000AF919F918F917F916F915F914F913F911F
:1001A0002F910F900FBE0F901F901895CF93DF9354
:1001B000DC01EC018A81282F33272530310509F431
:1001C00074C0263031059CF422303105C9F123304A
:1001D000310524F42130310519F1C9C0233031052E
:1001E00009F442C02430310509F44EC0C0C02830A3
:1001F000310509F494C0293031054CF4263031051D
:1002000009F471C02730310509F47DC0B0C0293030
:10021000310509F494C02A30310509F497C0A7C00C
:10022000FD01339682E0ED018B8381E081838EE6D0
:1002300094E09383828384E08A8385E090E09AC08F
:10024000ED01EC81E83008F0E0E081E0ED018A8327
:10025000FF27EE0FFF1FE050FF4F0190F081E02DD0
:1002600080818B83C90186C0FD013496ED018C81AC
:1002700031812281883008F080E0E82FFF27EE0FDF
:10028000FF1FE45EFE4F20C0ED01EC81E83008F076
:10029000E0E081E0ED018A83FF27EE0FFF1FE25FC0
:1002A000FE4F0190F081E02D35C0FD013496ED0147
:1002B0008C8131812281883008F080E0E82FFF278F
:1002C000EE0FFF1FE25FFE4FA081B181932F90954B
:1002D0008C9189238C930190F081E02D23238081E0
:1002E000822B808341C0FD01948187B1807C892B62
:1002F00087B9369A3699FECF82E0ED018A8384B1C0
:100300008B8385B118C0FD018481E82FFF2781E030
:10031000ED018A8380818B8382E090E02BC0FD0118
:100320008481E82FFF272081318182E0ED018A83DB
:100330002B83832F99278C8383E090E01BC0FD01E2
:100340008481E82FFF27ED018D81CBCFFD0134960D
:10035000ED018C81A82FBB2782819381892F99275A
:100360002281FD0181832C9380E090E003C0CD01C8
:100370000E943902DF91CF910895E0912D01F09113
:100380002E0109950895E0912F01F091300188E345
:1003900092E0099599270895CF93DF93EC0144E00B
:1003A00050EF61E070E06BBFFA0187919691875042
:1003B000904BA9F446E050EF61E070E06BBFFA01AA
:1003C00087919691AC0166277727440F551F661FCA
:1003D000771F6BBFFA0187919691039718F480E01D
:1003E00090E044C04E5F5F4F6F4F7F4F26E030E09C
:1003F0008DE291E00E94F1029091720086E3E8E3C1
:10040000F2E0282F11922A95E9F78093380281E0D3
:100410008093390280933A0210923C0210923B0280
:10042000D0933E02C0933D0281B38C7F81BB82B3E7
:100430008C7F82BB80E28093700080917400846026
:100440008093740080917400806880937400809120
:100450007400816080937400809174008064809344
:1004600074009E7F9093720081E090E0DF91CF91C5
:100470000895E0913101F0913201BC0183E391E0F4
:1004800009950895009731F0A4E0B0E01197F1F7D5
:100490000197D1F70895009731F0A0EABFE01197D6
:1004A000F1F70197D1F70895CF93C82F882331F042
:1004B00084E690E00E944202C150D1F7CF910895A6
:1004C000CF93C82F882331F08AE090E00E94420247
:1004D000C150D1F7CF910895CF93C82F882331F021
:1004E00084E690E00E944B02C150D1F7CF9108956D
:1004F000CF93C82F882331F08AE090E00E944B020E
:10050000C150D1F7CF910895CF93C82F882331F0F0
:1005100081E090E00E944B02C150D1F7CF91089545
:100520001F920F920FB60F9211248F939F93809179
:100530002C018F5F80932C018A3058F010922C018F
:1005400080912A0190912B01019690932B01809329
:100550002A0186E082BF9F918F910F900FBE0F906E
:100560001F90189584E083BF12BE81E087BF789406
:10057000089520912A0130912B0180912A019091B8
:100580002B0182179307C9F308959FEF9BBB1ABAFB
:1005900098BB80E187BB95BB14BA92BB11BA93B9E3
:1005A00012B810926200109261009093650088E189
:1005B0008093640010BE1092900089E189B91BB845
:1005C00088E98AB98EE08093950087EC86B980E44B
:1005D00087B986B1877C11F03699FECF0E94B202AE
:1005E00008956BBFFA01DC0102C007900D92215003
:0605F0003040D8F7089529
:1005F60039003600330030002100200063003A0045
:100606003700340031002200610064003B003800EE
:0A0616003500320023006200650089
:00000001FF
